:020000040000FA
:10040000EE2B0800080008000900200030163D000F
:1004100010185E2B901D08000F0887009011200017
:100420007839031DA232071973322008343A031DAC
:100430006732A001A401B101B013B81BB01739088D
:10044000FB3E03194432090B10323B0B063283305A
:10045000B3008830B20012303132090B4A32833097
:10046000B3009A30B200433029320903090B083235
:1004700030080139A63EB2008330B30001301E328D
:10048000090B06323A08B0000830E422AC001F32F3
:10049000E93E031D07323D000E122000A413A50102
:1004A00000301C32090B06328330B300E730B20053
:1004B00007300432090B1D32B0140730B100BF08F9
:1004C000031D05323E02031802323E08B1003D0012
:1004D0000E122000B81F09329422483083222409CA
:1004E00040390838A400A4170800A413A5010C3053
:1004F000F5333D000E1220000C3072220C30033216
:10050000200940390838A0000830A100A0170800D1
:10051000B01F02329422E3333908053A031D080064
:100520003A083D0096000800A501B108031908002B
:100530003208840033088500383086008701A51909
:10054000053212001E00A50AB10BF9330408B200EF
:100550000508B30008002000AC1BFE33AD002C09D9
:1005600040390838AC00AC170800071A0800071D0E
:100570000432B01AAC1B080001002908301E0332F7
:10058000022280311D3203191B323013E922301F41
:1005900013328700850060308400230015140000AA
:1005A000000013081A0014081A00910A870BF6338A
:1005B0004030AB22030103322100B0000130AB22F6
:1005C0002000280940390838A8004030A900A817A1
:1005D00048344108870040088600A90B0532523A8A
:1005E000031D0234B0160134A90B023201080800C1
:1005F000A90B0332420881000134A90B1B322300EE
:10060000950107089200871B151706089100200026
:100610001F39031D023442084308523A031D0232B7
:1006200030172034173A031D013423001516151511
:10063000472301343C30A906031D023420308400D6
:1006400085002300951615152030870012008607B7
:10065000930012008607940087030319033247238F
:10066000910AF43395128608031D03344723871635
:1006700015140000000011001402031D04341100C1
:100680001302031D04349103870BF23301345530F8
:100690009600AA3096009514000000000800210082
:1006A000FC3099001A095139031DFC3327009030A2
:1006B0009B005E233D008E018E1508003D009001D9
:1006C00014309100850120308400860003011A0057
:1006D000860BFD333D000E1796010E120E13901D72
:1006E000033290114E23FB33163098001E309900D0
:1006F0001A309A0020001830A200A6002030AA006C
:100700006030AE002030A300A700AB00AF007E2A0F
:10071000123401340034023402340034003408341A
:10072000D8340434DA34EF34013400340034003483
:1007300000340134093402344334003402340134C7
:100740000034803432340934043400340034013449
:1007500002340234013400340534243400341034BB
:10076000013404342434023402340534243406348D
:1007700000340134053424340134033401340734A3
:100780000534823403340834003402340934043428
:100790000134003402340A340034003400340734A5
:1007A0000534013402344034003400340734053455
:1007B00081340234403400340034A1342034003415
:1007C0000034003400340234003403340034803404
:1007D0002534003400340034003408344F23210021
:1007E0002B308C0037308E0020003B309B000430D3
:1007F0009C002C0094011E309500C030960005220C
:06080000FE330800103475
:00000001FF
